:020000040800F2
:1000000000060020A1020008791000087D100008F9
:10001000D11000087D100008A5100008A3020008F8
:10002000A3020008A3020008A3020008292A00086E
:10003000A3020008A3020008A3020008A30200080C
:10004000A3020008A3020008A3020008A3020008FC
:10005000A3020008A3020008353E0008613E000824
:100060008D3E0008B93E0008E53E0008A3020008E6
:10007000A3020008A3020008A3020008A3020008CC
:10008000A3020008A3020008A3020008A3020008BC
:10009000A3020008A3020008A3020008113F000801
:1000A000A3020008A3020008A3020008A30200089C
:1000B000A3020008A3020008A3020008A30200088C
:1000C000A3020008A3020008A3020008A30200087C
:1000D000A302000861110008A3020008A30200089F
:1000E000793F0008A3020008A3020008A302000849
:1000F000A3020008A3020008A3020008A30200084C
:10010000A3020008A3020008C13A0008A3020008E5
:10011000A3020008A3020008A3020008A30200082B
:10012000A3020008A3020008A3020008A30200081B
:10013000A3020008A3020008A3020008A30200080B
:10014000A3020008A3020008A3020008A3020008FB
:10015000A3020008A3020008A3020008A3020008EB
:10016000A3020008A3020008A3020008A3020008DB
:10017000A302000861350008A3020008A3020008DA
:10018000A3020008A3020008A3020008A3020008BB
:10019000A3020008A3020008A3020008A3020008AB
:1001A000A3020008A3020008A3020008A30200089B
:1001B000A3020008A3020008A3020008A30200088B
:1001C000A3020008A3020008A3020008A30200087B
:1001D000A30200084D350008A3020008A30200088E
:1001E000A3020008A3020008A3020008A30200085B
:1001F000A3020008A3020008A3020008A30200084B
:10020000A3020008A3020008A3020008A30200083A
:10021000A3020008A3020008A3020008A30200082A
:10022000A3020008A3020008A3020008A30200081A
:10023000A3020008A3020008A3020008A30200080A
:10024000A3020008A3020008A3020008A3020008FA
:10025000A3020008A3020008A3020008A3020008EA
:10026000A3020008A3020008A3020008A3020008DA
:10027000A3020008A3020008A3020008A3020008CA
:10028000A3020008A3020008A3020008A3020008BA
:10029000A3020008A3020008A3020008A3020008AA
:1002A00002E000F000F8FEE772B6394880F30888F3
:1002B000384880F3098838484EF60851CEF20001DC
:1002C000086040F20000CCF200004EF63471CEF22D
:1002D00000010860BFF34F8FBFF36F8F40F2000043
:1002E000C0F2F0004EF68851CEF200010860BFF374
:1002F0004F8FBFF36F8F4FF00000E1EE100A4EF604
:100300003C71CEF200010860062080F31488BFF330
:100310006F8F02F0C7FB03F051FB4FF055301F49C0
:100320001B4A91423CBF41F8040BFAE71C49194AA9
:1003300091423CBF41F8040BFAE71A491A4A1B4B99
:100340009A423EBF51F8040B42F8040BF8E7002034
:100350001749184A91423CBF41F8040BFAE702F0F2
:10036000E5FB03F09FFB144C144DAC4203DA54F848
:10037000041B8847F9E700F03FF8114C114DAC42DF
:1003800003DA54F8041B8847F9E702F0CDBB0000FC
:1003900000060020002600200000000800000020C9
:1003A00000060020D8430008002600204426002034
:1003B0004826002060370020A0020008A0020008A4
:1003C000A0020008A00200082DE9F04F2DED108AD0
:1003D000C1F80CD0D0F80CD0BDEC108ABDE8F08F7D
:1003E000002383F311882846A047002001F078FFFE
:1003F00001F094FE00DFFEE738B51F4C0123002515
:1004000023700423A57063701A23E570257165714C
:10041000A571E57125726572A372E57200F008FDA1
:1004200020B10E2325726572A372E57202F0BEFA46
:10043000044602F0F3FA0546D0B9104B9C4219D09D
:1004400001339C4241F2883412BF05460024012545
:10045000002002F0B5FA0DB100F05AF800F0B2FD3C
:1004600000F020FC204600F013F900F051F8F9E705
:100470000024EDE70446EBE748260020010007B022
:1004800008B500F08DFBA0F120035842584108BD8B
:10049000054B07B51B88022101A8ADF8043000F018
:1004A000EBFB03B05DF804FB8040000810B520238F
:1004B00083F311881248C3680BB101F097FF002342
:1004C000104A4FF47A710E4801F054FF002383F371
:1004D00011880D4C236813B12368013B23606368C6
:1004E00013B16368013B6360084B1B7833B96368E1
:1004F00023B9022000F0D6FC3223636010BD00BF98
:1005000054260020AD040008702700206826002033
:10051000554B56492DE9F04153F8042F013201D1D2
:10052000BDE8F0818B42F7D1514C524B22689A4280
:1005300040F29880504B9B6803F1006303F5003351
:100540009A4280F08F80002000F0D6FB02204B4BB7
:10055000187000F09DFC4A4BD3F8E8200022C3F845
:10056000E820D3F81011C3F81021D3F81011D3F8F4
:10057000EC10C3F8EC20D3F81411C3F81421D3F80D
:100580001411D3F8F010C3F8F020D3F81811C3F801
:100590001821D3F81811D3F8801041F00061C3F886
:1005A0008010D3F8801021F00061C3F88010D3F8D8
:1005B0008010D3F8801041F00071C3F88010D3F898
:1005C000801021F00071C3F88010D3F8803072B62B
:1005D0002C4B2D490B601D682468BFF34F8FBFF370
:1005E0006F8F2A4BC3F88420BFF34F8F5A6922F4D0
:1005F00080325A61BFF34F8FD3F8802043F6E07EFC
:10060000C2F3C906C2F34E32B707520102EA0E081E
:1006100038463146013948EA000C00F14040B1F15A
:10062000FF3FC3F874C2F5D1203A12F1200FEDD18B
:10063000BFF34F8FBFF36F8FBFF34F8FBFF36F8F3A
:100640005A6922F400325A610022C3F85022BFF3E3
:100650004F8FBFF36F8F202383F31188AD4685F34F
:1006600008882047BDE8F081FCFF01081C00020853
:1006700004000208FFFF0108482600206826002029
:10068000004402580000020808ED00E000ED00E020
:100690002DE9F04F99B0B34C2022FF21019010A812
:1006A000A66800F031FCB04AA3461378A3B9012133
:1006B000AE481170C360202383F31188C3680BB167
:1006C00001F094FE0023AA4A4FF47A71A74801F082
:1006D00051FE002383F31188019B13B1A54B019AAE
:1006E0001A600023A44AA349019F99461C461D464F
:1006F000984613704B600292012000F0C9FB002F56
:1007000000F012829B4B1B68002B40F00D8219B049
:10071000BDE8F08F0220FFF7B3FE002840F0FB8118
:10072000019BB9F1000F08BF1F46944B1B880221A3
:100730000BA8ADF82C3000F09FFADDE74FF47A708B
:1007400000F02EFA031E0393EADB0220FFF798FE67
:1007500082460028E4D0039B581E042800F2DD8165
:10076000DFE800F0030E1114170018A80523042178
:1007700040F8343D00F080FA54464FF0000856E04F
:1007800004217848F6E704217D48F3E704217D48F9
:10079000F0E71C242046043400F0B0FA04210B904A
:1007A0000BA800F069FA2C2CF4D1E5E7002DB7D0A6
:1007B000002CB5D00220FFF763FE0546002800F0AC
:1007C000AF8101206C4C00F097FA4FF00009022035
:1007D000207000F05DFB5FFA89FA504600F09CFA49
:1007E000074658B1504609F1010900F0A5FA002862
:1007F000F1D12C46A9460027634B97E701233E46DB
:100800000220237000F03AFBDBF808309E4206D24B
:10081000304600F073FA0130EBD10436F4E70026DD
:10082000029BA9462C461E703746524B5E6000F074
:10083000BFFB15B1002C18BF0027FFF729FE5BE7AF
:10084000002D3FF46DAF002C3FF46AAF0220029BF5
:10085000187000F01DFB322000F0A2F9B0F1000A80
:10086000C0F25E811AF0030540F05A8106EB0A03DC
:10087000DBF80820934200F25381BAF5807F00F242
:100880004F8155450DDA4FF47A7000F089F90490E4
:10089000049B002BC0F24481049B3C4AAB540135BD
:1008A000EFE7C820FFF7ECFD0546002800F038818F
:1008B0001F2E11D8C6F1200410AB26F003003349D7
:1008C0005445184428BF5446224600F0F5FA224603
:1008D000FF212E4800F018FB4FEAAA0A2B493046A8
:1008E0005FFA8AF200F018FB0446002800F01A8133
:1008F00006EB8A0605469AE70220FFF7C1FD0028AD
:100900003FF40EAF00F032FA00283FF409AF4FF089
:10091000000A5346DBF8082092451CD2BAF11F0F9B
:1009200012D8109A01320FD02AF0030218A90A44F3
:1009300052F8202C0B92184604220BA90AF1040A43
:1009400000F0DAFB0346E5E75046039300F0D6F9E2
:10095000039B0B90EFE718A8042140F84C3D00F0F2
:100960008BF964E7482600206C27002054260020DD
:10097000AD0400087027002068260020824000088F
:100980004C26002050260020844000086C260020C1
:1009900018A80023642140F8343D00F039F90028FC
:1009A0007FF4BEAE0220FFF76BFD00283FF4B8AE27
:1009B0000B9800F0D3F918AB43F8480D0421184602
:1009C000CDE718A80023642140F8343D00F020F959
:1009D00000287FF4A5AE0220FFF752FD00283FF467
:1009E0009FAE0B9800F0BCF918AB43F8440DE5E757
:1009F0000220FFF745FD00283FF492AE00F0C6F953
:100A000018AB43F8400DD9E70220FFF739FD002865
:100A10003FF486AE0BA9142000F0BEF9824618A858
:100A2000042140F83CAD00F027F951460BA896E7A9
:100A3000322000F0B5F8B0F1000AFFF671AE1AF0FE
:100A4000030F7FF46DAE0AEB0803DBF80820934236
:100A50003FF666AE0220FFF713FD00283FF460AEBC
:100A60002AF0030AC244D0453FF4E1AE404608F103
:100A7000040800F043F904210A900AA800F0FCF8E9
:100A8000F1E74FF47A70FFF7FBFC00283FF448AE23
:100A900000F06CF900283FF4AFAE109B01330CD08E
:100AA000082210A9002000F037FA00283FF4A4AE75
:100AB0002022FF2110A800F027FAFFF7E9FC3748B1
:100AC00001F014FC23E6002D3FF42AAE002C3FF485
:100AD00027AE18A80023642140F8343D00F098F8B0
:100AE000824600287FF41CAE0220FFF7C9FC0028D4
:100AF0003FF416AE0390FFF7CBFC41F28830574627
:100B000001F0F4FB0B9800F097FA00F051FA039B08
:100B10001C461D46F0E5054689E64FF00008FFE556
:100B20002546FDE52C4667E6002000F039F80490E4
:100B3000049B002BFFF6E3AD012000F09FF9049B1E
:100B4000213B122B3FF6D8AD01A252F823F000BF93
:100B5000150700083D070008AD070008F906000862
:100B6000F9060008F906000841080008310A0008E3
:100B7000F908000891090008C3090008F1090008F4
:100B8000F9060008090A0008F9060008830A0008A7
:100B90002F080008F9060008C70A0008A08601000F
:100BA0002DE9F3474FF47A75002402AE154F454303
:100BB000DFF8588006F8014D97F900305FFA84F9A4
:100BC0005A1C01D0A34212D158F824000122314608
:100BD0000368D3F820A02B46D047012807D10A4B41
:100BE0009DF8070083F8009002B0BDE8F08701345B
:100BF000022CE1D14FF4FA7001F078FB4FF0FF3096
:100C0000F2E700BF00260020BC2700209840000823
:100C10002DE9F0474FF47A7506460024134F4D43F3
:100C2000DFF8508097F900305FFA84F95A1C01D040
:100C3000A34210D158F82400042231460368D3F8A7
:100C400020A02B46D047042805D1094B002083F86B
:100C50000090BDE8F0870134022CE3D14FF4FA7024
:100C600001F044FB4FF0FF30BDE8F0870026002084
:100C7000BC27002098400008074B30B41A78074B77
:100C800053F822400A46014623682046DD69044B9A
:100C9000AC4630BC604700BFBC270020984000082D
:100CA000A0860100F8B5104C0025104E01F066FD3D
:100CB0000F4F20703068237883420CD800250D4EEA
:100CC0002078013801F056FD23780544013BB542F8
:100CD0002370F5D9F8BD01F04DFD336805440133AB
:100CE000BD423360E6D9E9E7BD2700207827002020
:100CF000FFFF0100FFFF030001F00CBE00F10060E8
:100D000000F500300068704700F10060920000F5C7
:100D1000003001F08FBD0000054B1A68054B1B78B1
:100D20009B1A834202D9104401F024BD0020704771
:100D300078270020BD27002038B5074D04462868D5
:100D4000204401F01DFD28B928682044BDE8384042
:100D500001F028BD38BD00BF782700200020704773
:100D6000014BC058704700BF00E8F11F064991F8D9
:100D7000243033B100230822086A81F82430FFF7B9
:100D8000C3BF0120704700BF7C270020014B1868BB
:100D9000704700BF0010005C234BF0B5234C1B686C
:100DA0002788C3F30B0665681B0C94F90820BE4224
:100DB00028D0A789BE4206D101220C2505FB02449A
:100DC000656894F9082041F20104A3421CD041F265
:100DD0000304A3421AD042F20104A34218D042F203
:100DE0000304A34208BF5622441E013D0B460C4497
:100DF000A34217D215F9016F581C5EB1034600F8E3
:100E0000016CF5E70022D8E75A22EDE75922EBE71B
:100E10005822E9E72C2584421D7001D9981C5A708C
:100E2000401AF0BD1846FBE70010005C04260020C5
:100E3000104B41F201015B888B429AB211D041F212
:100E400003018B420FD042F201039A420DD042F2CD
:100E500003039A420BD10323074A02EB8303D8789A
:100E600070470023F8E70123F6E70223F4E70020A8
:100E7000704700BF0010005C88400008022803D1C2
:100E80004FF00052014B9A61704700BF00080258B2
:100E9000022803D14FF40052014B9A61704700BF02
:100EA00000080258022804D1024A536983F400530F
:100EB0005361704700080258002310B5934203D0D5
:100EC000CC5CC4540133F9E710BD000030B5441EBA
:100ED00014F9010F0B4658B193F9005001318542C6
:100EE00006D11AB993F90020801A30BD013AEFE714
:100EF000002AF7D1104630BD02460346981A13F96E
:100F0000011B0029FAD1704702440346934202D0E4
:100F100003F8011BFAE770472DE9F047234C05461B
:100F20008846174694F8243083BB2E46DFF87C9021
:100F3000C7B394F824302BB92022FF2148462662FB
:100F4000FFF7E2FF94F824004146C0F1080504EBE6
:100F50008000BD4228BF3D465FFA85FAAD00A7EB91
:100F60000A072A462E44FFF7A7FF94F82430A84426
:100F7000FFB29A445FFA8AFABAF1080F84F824A003
:100F8000D6D1FFF7F3FE0028D2D108E0266A06EB9F
:100F90008306B042CAD0FFF7E9FE0028C5D1002081
:100FA000BDE8F0870120BDE8F08700BF7C27002066
:100FB000024B1A78024B1A70704700BFBC27002002
:100FC0000026002038B5164C164D204600F02CFCAB
:100FD0002946204600F054FC2D681348D5F890208F
:100FE000D2F8043843F00203C2F8043801F07EF965
:100FF0000E49284600F054FDD5F890200C48D2F850
:1010000004380C49A04223F00203C2F804384FF41C
:10101000E1330B6003D0BDE8384000F063BB38BD5E
:10102000E82E0020A041000840420F00C8410008FF
:1010300040280020A427002038B50B4B05461A781D
:101040000A4B53F822400A4B9C420CD0094B00211A
:1010500018221846FFF758FF056001462046BDE8F4
:10106000384000F03FBB38BDBC2700209840000846
:10107000E82E0020A4270020FEE7000000B59BB06A
:10108000EFF3098168226846FFF716FFEFF3058347
:10109000034B9A6B9A6A9A6A9A6A9A6A9B6AFEE703
:1010A00000ED00E000B59BB0EFF3098168226846CF
:1010B000FFF702FFEFF30583044B9A6B9A6A9A6A73
:1010C0009A6A9A6A9A6A9B6AFEE700BF00ED00E09E
:1010D00000B59BB0EFF3098168226846FFF7ECFE8C
:1010E000EFF30583034B5A6B9A6A9A6A9A6A9A6A73
:1010F0009B6AFEE700ED00E030B50A44074D9142DF
:101100000BD011F8013B09245840013CF7D040F3C3
:1011100000032B4083EA5000F7E730BD2083B8ED91
:10112000002304491A465A50C81808334260802BDD
:10113000F9D17047C0270020024A136843F0C0036A
:101140001360704700100140044B5A6810439A68BE
:1011500058600AB1181D1047704700BF4028002092
:101160002DE9F84F414EF56D2F68EC6921072C628F
:1011700019D014F0080F0CBF00208020E20748BFF0
:1011800040F02000A3074FF0200348BF40F040008C
:10119000610748BF40F4807083F31188FFF7D4FFE4
:1011A000002383F31188E20509D5202383F31188F6
:1011B0004FF40070FFF7C8FF002383F311884FF04E
:1011C0002009DFF8A8A04FF0000B14F0200832D15E
:1011D0003B0615D54FF02009DFF894A020060FD567
:1011E00089F31188504600F0F1F9002830DA082020
:1011F000FFF7AAFF27F080032B60002383F31188F9
:1012000079060DD562060BD5202383F31188F26C85
:10121000336D9A4201D1336C03BB002383F31188F1
:10122000E30604D5B26E13690BB150699847BDE867
:10123000F84F01F009BC89F31188AB8C504696F841
:101240006410194000F05CFA8BF31188EC69BCE77C
:1012500080B2288588F31188EC69BFE727F0400742
:101260001020FFF771FF2F60D7E700BF4028002054
:101270007828002013B5104C204600F027FA04F11E
:101280001400009400234FF400720C4900F0E8F8B9
:1012900004F1380000944FF40072094B094900F042
:1012A00061F9094B0C212520E365084B236602B048
:1012B000BDE8104000F05EB840280020AC280020B7
:1012C00039110008AC2A00200010014000E1F505AA
:1012D000254B002908BF1946037C012B816630B5D8
:1012E00011D1224B98420ED1214BD3F8F02042F07D
:1012F0001002C3F8F020D3F8182142F01002C3F80E
:101300001821D3F818310A68036EC46D03EB520339
:10131000B3FBF2F34A68150442BF23F0070503F05C
:10132000070343EA4503E3608B6843F040036360CF
:10133000CB68510543F00103A36042F4967343F078
:10134000010323604FF0FF33236205D512F0102212
:1013500005D0B2F1805F04D080F8643030BD7F23C7
:10136000FAE73F23F8E700BFBC4000084028002010
:101370000044025800F1604300F01F0209014009D7
:1013800003F56143C9B2800083F80013012300F123
:101390006040934000F56140C0F8803103607047C1
:1013A000F8B51546826804460B46AA4200D2856805
:1013B000A1692669761AB54207D218462A46FFF770
:1013C0007BFDA3692B44A3610DE011D9AF1B32460D
:1013D0001846FFF771FD3A46E1683044FFF76CFDAF
:1013E000E2683A44A261A36828465B1BA360F8BD8B
:1013F00018462A46FFF760FDE368E4E783689342F6
:101400002DE9F04104460F46154600D28568606913
:101410002669361AB54207D22A463946FFF74CFDEF
:1014200063692B4463610EE013D9A5EB06083246CD
:101430003946FFF741FD4246B919E068FFF73CFD28
:10144000E26842446261A36828465B1BA360BDE872
:10145000F0812A463946FFF72FFDE368E2E70000F6
:1014600010B50A440024C361029B006040608460A0
:10147000C160816141610261036210BD08B582698A
:101480004369934201D1826882B9826801328260E5
:101490005A1C42611970426903699A4201D3C368B8
:1014A0004361002100F03EFF002008BD4FF0FF30F7
:1014B00008BD000070B5202304460E4683F3118852
:1014C000A568A5B1A368A269013BA360531CA361F1
:1014D00015782269934224BFE368A361E3690BB1E5
:1014E00020469847002383F31188284670BD314673
:1014F000204600F007FF0028E2DA85F3118870BD6E
:101500002DE9F74F05460F4690469A46D0F81C90B5
:10151000202686F311884FF0000B144664B1224652
:1015200039462846FFF73CFF034668B9514628462E
:1015300000F0E8FE0028F1D0002383F31188A8EB27
:10154000040003B0BDE8F08FB9F1000F03D00190A3
:101550002846C847019B8BF31188E41A1F4486F381
:101560001188DBE7C160816141611144C361009B67
:10157000006040608260016103627047F8B5044614
:101580000E461746202383F31188A568A5B1A368EA
:10159000013BA36063695A1C62611E702369626922
:1015A0009A4224BFE3686361E3690BB12046984720
:1015B000002080F31188F8BD3946204600F0A2FED5
:1015C0000028E2DA85F31188F8BD000083694269DA
:1015D0009A4210B501D182687AB98268013282607C
:1015E0005A1C82611C7803699A4201D3C3688361E3
:1015F000002100F097FE204610BD4FF0FF3010BDD7
:101600002DE9F74F05460F4690469A46D0F81C90B4
:10161000202686F311884FF0000B144664B1224651
:1016200039462846FFF7EAFE034668B95146284680
:1016300000F068FE0028F1D0002383F31188A8EBA6
:10164000040003B0BDE8F08FB9F1000F03D00190A2
:101650002846C847019B8BF31188E41A1F4486F380
:101660001188DBE7026843681143016003B1184742
:10167000704700001430FFF743BF00004FF0FF3306
:101680001430FFF73DBF00003830FFF7B9BF00004E
:101690004FF0FF333830FFF7B3BF00001430FFF7CF
:1016A00009BF00004FF0FF311430FFF703BF000007
:1016B0003830FFF763BF00004FF0FF323830FFF7DC
:1016C0005DBF000000207047FFF7D4BD044B0360EE
:1016D000002343608360C36001230374704700BF2D
:1016E000D440000810B52023044683F31188FFF787
:1016F000EFFD02232374002383F3118810BD000043
:1017000038B5C36904460D461BB904210844FFF7E8
:10171000A9FF294604F11400FFF7B0FE002806DAFD
:10172000201D4FF48061BDE83840FFF79BBF38BDF6
:10173000026843681143016003B118477047000015
:1017400013B5446BD4F894341A681178042915D170
:10175000217C022912D11979012312898B4013426D
:101760000CD101A904F14C0002F02CF8D4F89444F7
:101770000246019B2179206800F0EAF902B010BD11
:10178000143001F0AFBF00004FF0FF33143001F010
:10179000A9BF00004C3002F081B800004FF0FF33C9
:1017A0004C3002F07BB80000143001F07DBF000027
:1017B0004FF0FF31143001F077BF00004C3002F0E1
:1017C0004DB800004FF0FF324C3002F047B8000037
:1017D000D0F8942438B5136805461978042901D047
:1017E000012038BD017C0229FAD1127901205C89DF
:1017F00090400440F4D105F1140001F00FFF0246BF
:101800000028EDD0D5F894544FF480732868697996
:1018100000F08CF9204638BD406BFFF7D9BF0000BF
:1018200000207047704700007FB5124B012502264B
:10183000044603600023057400F1840243602946D6
:101840008360C3600C4B0290143001934FF480739B
:10185000009601F0BFFE094B04F52372294601935F
:1018600004F14C004FF480730294009601F086FF5F
:1018700004B070BDFC4000081918000841170008AA
:101880000A68202383F311880B790B3342F8230075
:101890004B79133342F823008B7913B10B3342F8A1
:1018A00023000223C0F894140374002383F31188E7
:1018B0007047000038B5037F044613B190F85430E8
:1018C000ABB90125201D0221FFF732FF04F11400FE
:1018D00025776FF0010100F031FD84F8545004F1D8
:1018E0004C006FF00101BDE8384000F027BD38BD65
:1018F00010B5012104460430FFF71AFF00232377B7
:1019000084F8543010BD000038B50446002514306A
:1019100001F078FE04F14C00257701F047FF201D0F
:1019200084F854500121FFF703FF2046BDE83840FA
:10193000FFF74EBF90F8803003F06003202B19D1E1
:1019400090F88120212A0AD0222A4FF000030ED0DD
:10195000202A0FD1084A42670722826704E0064B1B
:101960004367072383670023C367012070474367EA
:101970008367F9E7002070471C260020D0F89434D4
:1019800037B51A680446117804291AD1017C022956
:1019900017D11979012312898B40134211D100F11B
:1019A0004C05284601F0C2FF58B101A9284601F0B4
:1019B00009FFD4F894440246019B2179206800F085
:1019C000C7F803B030BD000001F10B03F7B550F8C4
:1019D000234005460E46F4B1202383F3118805EB1E
:1019E0008607201D08214C34FFF7A2FEFB685B69C7
:1019F0001B6813B1204601F0F3FE01A9204601F057
:101A0000E1FE024648B1019B3146284600F0A0F8AD
:101A1000002383F3118803B0F0BDFB685A69126894
:101A2000002AF5D01B8A013B1340F1D105F1800259
:101A3000EAE70000133138B550F82140DCB120232B
:101A400083F31188D4F894241368527903EB82034A
:101A5000DB689B695D6845B104216018FFF768FE8B
:101A6000294604F1140001F0E3FD2046FFF7B0FE23
:101A7000002383F3118838BD7047000001F0DEB801
:101A8000012300F1300200F1500103700023436094
:101A900042F8043B8A42D361FAD103814381704703
:101AA00038B50446202383F31188002500F10C0388
:101AB00000F13002416043F8045B9342FBD12046C1
:101AC00001F0DEF80223237085F3118838BD000091
:101AD00070B500EB8103054650690E461446DA6086
:101AE00018B110220021FFF70FFAA06918B11022D7
:101AF0000021FFF709FA31462846BDE8704001F0A1
:101B0000D1B90000038900F13002002103F0010384
:101B10000381438903F00103438100F1100343F87B
:101B2000041B9342FBD101F055BA0000F0B401252B
:101B300000EB810447898D40E4683D43A4694581F9
:101B400023600023A2606360F0BC01F071BA000062
:101B5000F0B4012500EB810407898D40E4683D4322
:101B60006469058123600023A2606360F0BC01F01A
:101B7000E9BA0000022300F10C0200F1300110B5B7
:101B8000037004460023A0F8883080F88A3080F87B
:101B90008B300381438142F8043B8A42FBD184F8B5
:101BA0007030204601F012F963681B6823B12046AB
:101BB0000021BDE81040184710BD000002784368BE
:101BC00080F88C2005221B6802700BB10421184795
:101BD00070470000436890F88C201B6802700BB1BE
:101BE000052118477047000090F8703070B5044622
:101BF00013B1002380F8703004F18002204601F018
:101C00000DFA63689B6863BB94F8805015F060061A
:101C100015D194F8813005F07F0545EA032540F29F
:101C200002339D4200F00E815BD8022D00F0DC8073
:101C30003FD8002D00F08780012D00F0CF800021DB
:101C4000204601F0A3FC0021204601F093FC6368CC
:101C50001B6813B1062120469847062384F870308C
:101C600070BD204698470028CED094F8872094F87D
:101C7000863043EA0223A26F934238BFA36794F9E8
:101C80008030A56F002B4FF0200380F2FD80002DE7
:101C900000F0EC80092284F8702083F31188002181
:101CA000A36F626F2046FFF753FF002383F3118871
:101CB00070BDB5F5817F00F0B180B5F5407F49D0AA
:101CC000B5F5807FBBD194F88230012BB7D1B4F841
:101CD000883023F00203A4F888306667A667E667B9
:101CE000C3E740F201639D421ED8B5F5C06F3BD2F9
:101CF000B5F5A06FA3D1B4F88030B3F5A06F0ED1C5
:101D000094F88230204684F88A3001F0BDF8636888
:101D10001B6813B101212046984703232370002339
:101D20006367A367E367A0E7B5F5106F32D040F6AD
:101D300002439D4252D0B5F5006F80D104F18B0370
:101D40006367012324E004F18803E56763670223E6
:101D5000A3678AE794F88230012B7FF470AFB4F860
:101D6000883043F00203B6E794F885202046616886
:101D700094F884304D6843EA022394F8831094F871
:101D80008220A84700283FF45AAF4368636703687E
:101D9000A367A4E72378042B10D1202383F31188B1
:101DA0002046FFF7AFFE86F311886368032184F8AD
:101DB0008B601B6821700BB12046984794F88230E5
:101DC000002BACD084F88B300423237063681B682D
:101DD000002BA4D0022120469847A0E7374B636729
:101DE0000223A36700239DE794F88410204611F096
:101DF000800F01F00F010ED001F002F9012806D08A
:101E000002287FF41CAF2E4BA067636767E72D4B5A
:101E1000A567636763E701F0E5F8EFE794F88230C0
:101E2000002B7FF40CAF94F8843013F00F013FF4D3
:101E300076AF1A06204602D501F0C0FB6FE701F02D
:101E4000B1FB6CE794F88230002B7FF4F8AE94F885
:101E5000843013F00F013FF462AF1B06204602D519
:101E600001F094FB5BE701F085FB58E7142284F84E
:101E7000702083F311882B462A4629462046FFF717
:101E800055FE85F3118870BD5DB1152284F8702070
:101E900083F311880021A36F626F2046FFF746FE8F
:101EA00003E70B2284F8702083F311882B462A461F
:101EB00029462046FFF74CFEE3E700BF2C4100080F
:101EC000244100082841000838B590F870300446D5
:101ED000152B29D8DFE803F03E28282828283E289B
:101EE000280B293928282828282828283E3E90F819
:101EF000871090F88620836F42EA01229A4214D913
:101F0000C268128AB3FBF2F502FB15356DB92023C6
:101F100083F311882B462A462946FFF719FE85F3DD
:101F200011880A2384F8703038BD142384F8703087
:101F3000202383F31188002320461A461946FFF711
:101F4000F5FD002383F3118838BDC36F03B19847B3
:101F50000023E7E7002101F019FB0021204601F0F2
:101F600009FB63681B6813B10621204698470623C6
:101F7000D8E7000090F87020152A38B5044622D81A
:101F80000123934040F6416213421DD113F48015A2
:101F90000FD19B0217D50B2380F87030202383F3D9
:101FA00011882B462A462946FFF7D2FD85F3118872
:101FB00038BDC3689B695B682BB9C36F03B1984791
:101FC000002384F8703038BD002101F0DFFA0021D1
:101FD000204601F0CFFA63681B6813B10621204642
:101FE00098470623EDE70000024B00221B605B6070
:101FF0009A607047AC2C0020002382680374054B64
:102000001B6899689142FBD25A6803604260106075
:1020100058607047AC2C002008B5202383F311884A
:10202000037C032B05D0042B0DD02BB983F311882F
:1020300008BD436900221A604FF0FF334361FFF788
:10204000DBFF0023F2E790E80C001A60026853609F
:10205000F2E70000002382680374054B1B6899684F
:102060009142FBD85A680360426010605860704724
:10207000AC2C0020054B196908741868026853607D
:102080001A60186101230374FEF79EB9AC2C00207E
:102090004B1C30B5054687B00A4C10D0236901A807
:1020A000094A00F067F92846FFF7E4FF049B13B1E3
:1020B00001A800F09BF92369586907B030BDFFF70C
:1020C000D9FFF8E7AC2C00201920000838B50C4DDA
:1020D000044641612B6981689A68914203D8BDE842
:1020E0003840FFF789BF1846FFF786FF01232C61B0
:1020F000014623742046BDE83840FEF765B900BFAD
:10210000AC2C0020044B1A681B6990689B689842AD
:1021100094BF002001207047AC2C002010B5084C63
:10212000236820691A6854602260012223611A74AE
:10213000FFF790FF01462069BDE81040FEF744B963
:10214000AC2C0020FEE7000010B5194CFFF74CFF47
:1021500000F002F980221749204600F087F8012399
:1021600044F8180C0374144B144AD96821F4E06144
:102170000904090C0A431249DA60CA6842F0807205
:10218000CA60104A1049C2F8B01F116841F001013D
:1021900011601022DA77202283F82220002383F3B3
:1021A000118862B60948BDE8104000F081B800BF50
:1021B000D42C00203041000800ED00E00003FA05B7
:1021C000F0ED00E0001000E055CEACC5384100084D
:1021D0002DE9F84F1E4C4FF00008DFF87890656944
:1021E00004F11407D9F82430266AAA689E1B964287
:1021F0001CD34FF0200AAA68236AD5F80CB0B61A8F
:10220000134423622B68BB425F606361C5F80C8096
:1022100001D101F0B7FB88F311882869D8478AF308
:1022200011886569AB689E42E5D2DBE76269BA4214
:102230000CD0916823628E1B9660A86802282CBF80
:102240001818981CBDE8F84F01F0A2BBBDE8F88F44
:10225000AC2C0020000C0040034B59685A68521AFD
:102260009042FBD8704700BF001000E0826002225D
:1022700002740022427470478368A3F17C0243F821
:102280000C2C026943F83C2C426943F8382C074A6D
:1022900043F81C2CC268A3F1180043F8102C02224A
:1022A00003F8082C002203F8072C7047E10300080C
:1022B00010B5202383F31188FFF7DEFF00210446C9
:1022C000FFF704FF002383F31188204610BD0000B0
:1022D000024B1B6958610F20FFF7CCBEAC2C0020CD
:1022E000202383F31188FFF7F3BF000008B50146F0
:1022F000202383F311880820FFF7CAFE002383F30D
:10230000118808BD49B1064B42681B6918605A60C4
:10231000136043600420FFF7BBBE4FF0FF307047EF
:10232000AC2C00200368984206D01A680260506006
:1023300018465961FFF760BE7047000038B5044683
:102340000D462068844200D138BD036823605C607C
:102350004561FFF751FEF4E7054B03F114025A61A2
:102360009A614FF0FF32DA6100221A62704700BFB3
:10237000AC2C0020F8B5036102291A4B0646C26056
:1023800038BF02215C6A184B1A461F4652F8145F88
:1023900095420AD1586198611C6205604560816070
:1023A0000819BDE8F84001F0E3BA186AAB68241ACE
:1023B0000C1902D3E41A2D6804E09C4202D2204496
:1023C00001F0E6FAAB689C42F4D86B683560736044
:1023D0001E604FF0FF336E60B460A968091BA960EE
:1023E000FB61F8BD000C0040AC2C002010B41A4C6E
:1023F000234653F8141F814210D0416802680A60D6
:10240000026851609A424FF00001C16003D09368A6
:1024100081680B4493605DF8044B70470A680020A4
:102420009A4262615360C86003D15DF8044B01F0C9
:10243000A9BA936888680344206A9360074A526A7D
:10244000121A9342E7D9991A5DF8044B012998BFF3
:10245000931C184401F09CBAAC2C0020000C0040E6
:1024600000207047FEE70000704700004FF0FF308B
:1024700070470000022906D0032906D0012906482A
:1024800018BF0020704705487047032A9ABF0448C8
:1024900000EBC2000020704724420008D841000829
:1024A0002426002070B59AB006460846144601ADB1
:1024B000294600F095F82846FEF71EFDC0B2431CE1
:1024C0005B0086E8180023700323023404F8013C03
:1024D00000231946DAB20234904201D81AB070BD16
:1024E000EA5C013304F8011C04F8022CF2E7000056
:1024F00008B5202383F311880348FFF73FFA002330
:1025000083F3118808BD00BFE82E002010B50446F3
:10251000052916D8DFE801F016150316161D20232D
:1025200083F311880E4A0121FFF7D2FA20460D4AA3
:102530000221FFF7CDFA0C48FFF7E6F9002383F3F9
:10254000118810BD202383F311880748FFF7B2F9E3
:10255000F4E7202383F311880348FFF7C9F9EDE777
:10256000584100087C410008E82E002038B50C4D89
:102570000C4C2A460C4904F10800FFF793FF05F1C3
:10258000CA0204F110000949FFF78CFF05F5CA7271
:1025900004F118000649BDE83840FFF783BF00BFCB
:1025A000B033002024260020A8410008B2410008D2
:1025B000BD41000870B5044608460D46FEF79CFC78
:1025C000C6B22046013403780BB9184670BD3246B6
:1025D0002946FEF77BFC0028F3D1012070BD0000E6
:1025E0002DE9F84F05460C46FEF786FC2B49C6B28E
:1025F0002846FFF7DFFF2A492846FFF7DBFF08B12F
:102600001036F6B2632E0DD8DFF89080DFF8909088
:10261000244FDFF898A0DFF898B02E7846B92670DE
:10262000BDE8F88F29462046BDE8F84F01F020BDEF
:10263000252E2ED1072241462846FEF747FC70B9C9
:10264000DBF800300735073444F8073CBBF80430AA
:1026500024F8033C9BF8063004F8013CDDE708222F
:1026600049462846FEF732FC98B9A21C0E4B13F8D7
:10267000011F023209095345C95D02F8041C19788B
:1026800001F00F01C95D02F8031CF0D118340835C0
:10269000C3E7267001350134BFE700BF444200089C
:1026A000BD41000854420008FFE7F11F0BE8F11F8D
:1026B0004C420008BFF34F8F044B1A695107FCD1FD
:1026C000D3F810215207F8D1704700BF0020005204
:1026D00008B50D4B1B78ABB9FFF7ECFF0B4BDA6875
:1026E000D10704D50A4A5A6002F188325A60D3F8F9
:1026F0000C21D20706D5064AC3F8042102F188321C
:10270000C3F8042108BD00BF0E360020002000528F
:102710002301674508B5114B1B78F3B9104B1A69B3
:10272000510703D5DA6842F04002DA60D3F810218D
:10273000520705D5D3F80C2142F04002C3F80C2112
:10274000FFF7B8FF064BDA6842F00102DA60D3F80F
:102750000C2142F00102C3F80C2108BD0E36002006
:10276000002000520F289ABF00F58060400400202E
:10277000704700004FF40030704700001020704791
:102780000F2808B50BD8FFF7EDFF00F500330268FE
:10279000013204D104308342F9D1012008BD002068
:1027A00008BD00000F2810B504463FD8FFF782FF90
:1027B000FFF78EFF1E484FF0FF33072C4361C0F830
:1027C00014311DD80361FFF775FF230243F0240382
:1027D000C360C36843F08003C36003695A07FCD435
:1027E000FFF768FF2046FFF7BDFF4FF4003100F010
:1027F000F7F8FFF78FFF2046BDE81040FFF7C0BF96
:10280000C0F81031FFF756FFA4F108031B0243F094
:102810002403C0F80C31D0F80C3143F08003C0F829
:102820000C31D0F810315B07FBD4D9E7002010BD84
:10283000002000522DE9F84F40EA020305460E46FB
:102840001746DB0656D13446DFF8C090DFF8C0A04B
:10285000FFF73EFF3B1B33441F2B04D8FFF75AFF03
:102860000120BDE8F88F20222146284601F0F0FB28
:10287000002837D005F17843214A22489342224B61
:1028800098BF984603F5827392BFD346C8469B46CD
:10289000A3F1080388BF1846FFF70CFF4FF0FF3382
:1028A00004F11C01A5EB040ECBF80030036843F0E3
:1028B00002030360231FD8F8002012F0050FFAD19D
:1028C00053F8042F99424EF80320F4D1BFF34F8FF1
:1028D000FFF7F0FE4FF0FF33CBF80030036823F032
:1028E0000203036020222146284601F0B1FB20B1FB
:1028F000FFF710FF0020BDE8F88F20352034A9E74E
:10290000FFFF0F000C200052102000521021005237
:102910001420005210B5084C237828B153B9FFF7A2
:10292000D7FE0123237010BD23B12070BDE81040F5
:10293000FFF7F0BE10BD00BF0E3600200244043980
:10294000064BD2B210B5904200D110BD441C00B26B
:1029500053F8200041F8040FE0B2F4E7504000586B
:102960000F4B30B51C6F240405D41C6F1C671C6F03
:1029700044F400441C670B4C024404392368D2B26F
:1029800043F480732360084B904200D130BD441C57
:1029900051F8045F00B243F82050E0B2F4E700BF02
:1029A00000440258004802585040005807B5012220
:1029B00001A90020FFF7C2FF019803B05DF804FBF6
:1029C00013B50446FFF7F2FFA04206D002A9012288
:1029D000002041F8044DFFF7C3FF02B010BD000016
:1029E0000144BFF34F8F064B884204D3BFF34F8F90
:1029F000BFF36F8F7047C3F85C022030F4E700BF6D
:102A000000ED00E0034B1B685B0142BF0122024B5B
:102A10001A707047D04402580F360020014B1878C6
:102A2000704700BF0F360020064A536823F00103A9
:102A30005360EFF30983683383F30988002383F33A
:102A40001188704730EF00E010B5202383F3118820
:102A5000104B5B6813F4006318D0F1EE103AEFF3FB
:102A600009844FF0807344F84C3C0B4BDB6844F80E
:102A7000083CA4F1680383F30988FFF743FB18B10E
:102A8000064B44F8503C10BD054BFAE783F3118820
:102A900010BD00BF00ED00E030EF00E0F1030008E2
:102AA000F4030008F0B5BFF34F8FBFF36F8F1D4BDA
:102AB0000021C3F85012BFF34F8FBFF36F8F5A69D5
:102AC00042F400325A61BFF34F8FBFF36F8FC3F8E8
:102AD0008410BFF34F8FD3F8802043F6E076C2F323
:102AE000C904C2F34E32A507520102EA060E284677
:102AF00021464EEA0007013900F14040C3F86072F8
:102B00004F1CF6D1203A12F1200FEED1BFF34F8FB8
:102B10005A6942F480325A61BFF34F8FBFF36F8F0F
:102B2000F0BD00BF00ED00E0FEE70000084A094BE1
:102B300009498B4204D3094A0021934205D37047C7
:102B400052F8040F43F8040BF3E743F8041BF4E7CF
:102B500018440008603700206037002060370020EC
:102B6000D0F89430002230B51146D0F890409D68DE
:102B70004FF0FF3004EB421301329542C3F80019C5
:102B8000C3F81019C3F80809C3F8001BC3F8101BD9
:102B9000C3F8080BEED24FF00113C4F81C3830BD57
:102BA00000EB81032DE9F04FD3F80CE04F1C4FEA06
:102BB0004118DEF814403F03D4F800C06568D0F82F
:102BC000902065450AD30120D2F8343800FA01F18B
:102BD00023EA0101C2F83418BDE8F08FACEB05031D
:102BE000BEF81060B34228BF334602EB0806D6F8A1
:102BF0001869B6B2B3EB860F13D8A6683A44994663
:102C0000A6F1040A5AF804BFB9F1040FC2F800B0E3
:102C100002D9A9F10409F5E71E442B44A6606360BC
:102C2000CCE70020BDE8F08F890141F0200101616F
:102C300003699B06FCD41220FFF70EBB10B50A4CAB
:102C40002046FEF71DFF094BC4F89030084BC4F82E
:102C50009430084C2046FEF713FF074BC4F8903021
:102C6000064BC4F8943010BD103600200000084018
:102C70008C420008AC360020000004409842000856
:102C80000378012B70B505465DD1494BD0F89040D3
:102C9000984259D1474B0E216520D3F8D82042F0F5
:102CA0000062C3F8D820D3F8002142F00062C3F8D4
:102CB0000021D3F80021D3F8802042F00062C3F84D
:102CC0008020D3F8802022F00062C3F88020D3F85F
:102CD0008030FEF74FFB384BE360384BC4F80038C8
:102CE0000023D5F89060C4F8003EC02323604FF461
:102CF0000413A3633369002BFCDA01230C20336136
:102D0000FFF7AAFA3369DB07FCD41220FFF7A4FA15
:102D10003369002BFCDA00262846A660FFF720FF67
:102D20006B68C4F81068DB68C4F81468C4F81C68E1
:102D3000002B3AD1224BA3614FF0FF336361A368AC
:102D400043F00103A36070BD1E4B9842C8D1194BDC
:102D50000E214D20D3F8D82042F00072C3F8D820BD
:102D6000D3F8002142F00072C3F80021D3F800210B
:102D7000D3F8802042F00072C3F88020D3F880207E
:102D800022F00072C3F88020D3F88020D3F8D82036
:102D900022F08062C3F8D820D3F8002122F08062AC
:102DA000C3F80021D3F8003193E7074BC3E700BF16
:102DB0001036002000440258401400400300200256
:102DC000003C30C0AC360020083C30C0F8B5D0F82C
:102DD0009040054600214FF000662046FFF724FF93
:102DE000D5F8941000234FF001128F684FF0FF3098
:102DF000C4F83438C4F81C2804EB431201339F4252
:102E0000C2F80069C2F8006BC2F80809C2F8080BE2
:102E1000F2D20B68D5F89020C5F898306362102381
:102E20001361166916F01006FBD11220FFF714FA91
:102E3000D4F8003823F4FE63C4F80038A36943F4DF
:102E4000402343F01003A3610923C4F81038C4F8E9
:102E500014380B4BEB604FF0C043C4F8103B094BE8
:102E6000C4F8003BC4F81069C4F80039D5F89830AC
:102E700003F1100243F48013C5F89820A362F8BD53
:102E80006842000840800010D0F8902090F88A1026
:102E9000D2F8003823F4FE6343EA0113C2F8003885
:102EA000704700002DE9F0410EB20D4600EB860898
:102EB000D8F80C100F6807F00303022B53D0032B34
:102EC00053D03F4A3F4F012B18BF1746D0F89040D0
:102ED0004FEA451E002205F1100C04EB0E03C3F867
:102EE000102B8A69002A42D04A8A05F158033A43D6
:102EF0005B01E2500123D4F81C2803FA0CF31343BE
:102F0000C4F81C38A64400234A69CEF8103905F1EC
:102F10003F03002A3BD00A8A04EB8303898B920883
:102F2000012988BF4A43D0F89810561841EA024256
:102F30002946C0F8986020465A60FFF775FED8F819
:102F40000C301B8A43EA85531F4305F148035B019C
:102F5000E7500123D4F81C2803FA05F51543C4F8FB
:102F60001C58BDE8F081184FB0E7184FAEE704EBEE
:102F70004613D3F8002B22F40042C3F8002B0123A0
:102F8000D4F81C2803FA0CF322EA0303B8E704EB95
:102F900083030F4A04EB461629465A602046FFF782
:102FA00043FED6F80039012223F4004302FA05F566
:102FB000C6F80039D4F81C3823EA0505CFE700BF6E
:102FC00000800010008004100080081000800C10A9
:102FD00000040002D0F894201268C0F89820FFF78F
:102FE000BFBD00005831D0F8903049015B5813F450
:102FF000004004D013F4001F14BF012002207047CA
:103000004831D0F8903049015B5813F4004004D0A7
:1030100013F4001F14BF01200220704700EB810150
:10302000CB68196A0B6813604B68536070470000E7
:1030300000EB810330B5DD68AA691368D36019B964
:10304000402B84BF402313606B8A1468D0F8902013
:103050001C4402EB4110013C09B2B4FBF3F463439E
:10306000033323F0030343EAC44343F0C043C0F8EF
:10307000103B2B6803F00303012B0ED1D2F8083864
:1030800002EB411013F4807FD0F8003B14BF43F0F3
:10309000805343F00053C0F8003B02EB4112D2F8DA
:1030A000003B43F00443C2F8003B30BD2DE9F04142
:1030B000D0F8906005460C4606EB4113D3F8087B28
:1030C0003A07C3F8087B08D5D6F814381B0704D58F
:1030D00000EB8103DB685B689847FA072FD5D6F8C9
:1030E0001438DB072BD505EB8403D968CCB98B6981
:1030F000488A5E68B6FBF0F200FB12628AB9186873
:10310000DA6890420DD2121A83E81400202383F368
:10311000118821462846FFF78BFF84F31188BDE80C
:10312000F081012303FA04F26B8923EA02036B8125
:10313000CB6823B121462846BDE8F0411847BDE8D9
:10314000F081000000EB81034A0170B5DD68D0F822
:1031500090306C692668E66056BB1A444FF4002034
:10316000C2F810092A6802F00302012A0AB20ED13D
:10317000D3F8080803EB421410F4807FD4F8000958
:1031800014BF40F0805040F00050C4F8000903EB39
:103190004212D2F8000940F00440C2F800090122AE
:1031A000D3F8340802FA01F10143C3F8341870BDB2
:1031B00019B9402E84BF4020206020681A442E8A0E
:1031C000841940F00050013CB4FBF6F440EAC440DE
:1031D000C6E700002DE9F041D0F8906004460D46A6
:1031E00006EB4113D3F80879C3F80879FB071CD51F
:1031F000D6F81038DA0718D500EB8103D3F80CE0C5
:10320000DEF81430D3F800C0DA6894451BD2A2EB84
:103210000C024FF000081A60C3F80480202383F3E7
:103220001188FFF78FFF88F311883B0618D501231B
:10323000D6F83428AB40134212D029462046BDE8C8
:10324000F041FFF7ADBC012303FA01F2038923EA41
:1032500002030381DEF80830002BE6D09847E4E74C
:10326000BDE8F0812DE9F047D0F8905004466E6932
:10327000AB691E40F1046E6103D5BDE8F047FEF76F
:1032800079BC002E12DAD5F8003E9A0705D0D5F8A1
:10329000003E23F00303C5F8003ED5F8043820466D
:1032A00023F00103C5F80438FEF794FC330502D57A
:1032B0002046FEF783FCB7040CD5D5F8083813F088
:1032C000060FEB6823F470530CBF43F4105343F420
:1032D000A053EB60300704D56368DB680BB1204670
:1032E0009847F10200F1A180B2020BD5D4F890808A
:1032F00000274FF00109D4F89430F9B29B688B4253
:1033000080F0D280F3061AD5D4F890100A6AC2F37E
:103310000A1702F00F0302F4F012B2F5802F00F04A
:10332000EB80B2F5402F0AD104EB830301F5805105
:10333000DB68186A00231A469F4240F0D1803003B0
:10334000D5F8185835D5E90303D500212046FFF7F5
:10335000ADFEAA0303D501212046FFF7A7FE6B03AC
:1033600003D502212046FFF7A1FE2F0303D5032139
:103370002046FFF79BFEE80203D504212046FFF715
:1033800095FEA90203D505212046FFF78FFE6A02AC
:1033900003D506212046FFF789FE2B0203D507211E
:1033A0002046FFF783FEEF0103D508212046FFF7F3
:1033B0007DFE700340F1C780E90703D50021204658
:1033C000FFF708FFAA0703D501212046FFF702FFF8
:1033D0006B0703D502212046FFF7FCFE2F0703D51C
:1033E00003212046FFF7F6FEEE0603D50421204612
:1033F000FFF7F0FEA80603D505212046FFF7EAFEF9
:10340000690603D506212046FFF7E4FE2A0603D508
:1034100007212046FFF7DEFEEB0540F194802046B1
:103420000821BDE8F047FFF7D5BED4F890904FF0E3
:1034300000084FF0010AD4F894305FFA88F79B68CF
:10344000BB42FFF451AF09EB4713D3F8002902F454
:103450004022B2F5802F24D1D3F80029002A20DAA7
:10346000D3F8002942F09042C3F80029D3F800298C
:10347000002AFBDB3946D4F89000FFF7D5FB228900
:103480000AFA07F322EA0303238104EB8703DB68CC
:103490009B6813B139462046984739462046FFF7C6
:1034A0007FFB08F10108C6E708EB4112D2F8003BA8
:1034B00003F44023B3F5802F10D1D2F8003B002B4A
:1034C0000CDA628909FA01F322EA0303638104EB4F
:1034D0008103DB68DB680BB12046984701370AE7B8
:1034E00013F0030F00D10A68072B03F101039EBFFD
:1034F0000270120A01301FE704EB830301F58051CB
:10350000DA6890690268D0F808C04068A2EB000E43
:1035100000221046974208D1DB689B699A683A44BA
:103520009A605A6817445F6009E712F0030F00D1F0
:103530000868964502F1010282BF8CF80000000A7B
:103540000CF1010CE6E7BDE8F087000008B5034880
:10355000FFF788FEBDE80840FFF776BA1036002076
:1035600008B50348FFF77EFEBDE80840FFF76CBAD8
:10357000AC360020D0F8903003EB4111D1F8003B7D
:1035800043F40013C1F8003B70470000D0F89030BE
:1035900003EB4111D1F8003943F40013C1F80039AD
:1035A00070470000D0F8903003EB4111D1F8003B98
:1035B00023F40013C1F8003B70470000D0F89030AE
:1035C00003EB4111D1F8003923F40013C1F800399D
:1035D0007047000030B50433039C0172002104FBE6
:1035E0000325C361049B00600363059B4060C160C9
:1035F000426102618561046242628162C162436329
:1036000030BD00000022416AC260416101616FF07B
:1036100001018262C262FEF791BE00000369426945
:10362000934203D1C2680AB100207047181D704749
:10363000036919600021C2680132C260C269134483
:1036400082699342036124BF436A0361FEF76ABE45
:1036500038B504460D46E3683BB162690020131D8E
:103660001268A3621344E36238BD237A33B9294652
:103670002046FEF747FE0028EDDA38BD6FF0010066
:10368000FBE70000C368C269013BC36043691344A0
:1036900082699342436124BF436A4361002383628A
:1036A000036B03B11847704770B52023044683F3BA
:1036B0001188866A3EB9FFF7CBFF054618B186F33D
:1036C0001188284670BDA36AE26A13F8015B934231
:1036D000A36202D32046FFF7D5FF002383F31188AE
:1036E000EFE700002DE9F84F04460E469046994654
:1036F000202787F311880025AA46D4F828B0BBF10B
:10370000000F09D149462046FFF7A2FF20B18BF3F5
:1037100011882846BDE8F88FA16AA8EB050BE36A7B
:103720005B1A9B4528BF9B46BBF1400F1BD9334614
:1037300001F1400251F8040B914243F8040BF9D116
:10374000A36A403640354033A362A26AE36A9A42D4
:1037500002D32046FFF796FF8AF311884545D8D259
:1037600087F31188C9E730465A46FDF7A5FBA36ADF
:103770005E445D445B44A362E7E7000010B5029C31
:1037800004330172C36103FB0421002300608362E0
:10379000C362039B40600363049BC4604261026197
:1037A000816104624262436310BD0000026A6FF0EF
:1037B0000101C260426A4261026100228262C26209
:1037C000FEF7BCBD436902699A4203D1C2680AB1DF
:1037D00000207047184650F8043B0B60704700000B
:1037E000C3680021C2690133C3604369134482691D
:1037F0009342436124BF436A4361FEF793BD0000D7
:1038000038B504460D46E3683BB1236900201A1D14
:10381000A262E2691344E36238BD237A33B92946D0
:103820002046FEF76FFD0028EDDA38BD6FF001008D
:10383000FBE7000003691960C268013AC260C2690F
:10384000134482699342036124BF436A03610023E6
:103850008362036B03B118477047000070B52023E3
:1038600004460E4683F31188856A35B91146FFF781
:10387000C7FF10B185F3118870BDA36A1E70A36ADB
:10388000E26A01339342A36204D3E169204604391A
:10389000FFF7D0FF002080F3118870BD2DE9F84FAD
:1038A00004460D4691469A464FF0200888F3118849
:1038B0000026B346A76A4FB951462046FFF7A0FF3E
:1038C00020B187F311883046BDE8F88FA06AA9EBD4
:1038D0000603E76A3F1A9F4228BF1F46402F1BD9A5
:1038E00005F1400355F8042B9D4240F8042BF9D113
:1038F000A36A40364033A362A26AE36A9A4204D3C1
:10390000E16920460439FFF795FF8BF311884E4596
:10391000D9D288F31188CDE729463A46FDF7CCFA8B
:10392000A36A3D443E443B44A362E5E70269436920
:103930009A4203D1C3681BB9184670470023FBE7BE
:10394000836A002BF8D0043B9B1AF5D01360C36840
:10395000013BC360C3691A4483699A42026124BF70
:10396000436A0361002383620123E5E700F0BCB8EA
:10397000034B002258631A610222DA60704700BFCD
:10398000000C00400022014BDA607047000C004040
:10399000014B5863704700BF000C00404B68436008
:1039A0008B688360CB68C3600B6943614B690362BA
:1039B0008B6943620B6803607047000008B52C4BAD
:1039C00040F2FF712B48D3F888200A43C3F88820BF
:1039D000D3F8882022F4FF6222F00702C3F888207F
:1039E000D3F88820D3F8E0200A43C3F8E020D3F8C6
:1039F00008210A43C3F808211F4AD3F808311146A9
:103A0000FFF7CCFF1D4802F11C01FFF7C7FF1C4860
:103A100002F13801FFF7C2FF1A4802F15401FFF723
:103A2000BDFF194802F17001FFF7B8FF174802F116
:103A30008C01FFF7B3FF164802F1A801FFF7AEFFB4
:103A4000144802F1C401FFF7A9FF134802F1E00195
:103A5000FFF7A4FF114802F1FC01FFF79FFF104898
:103A600002F58C71FFF79AFFBDE8084000F016B927
:103A70000044025800000258A44200080004025802
:103A800000080258000C0258001002580014025896
:103A900000180258001C0258002002580024025846
:103AA0000028025808B500F0C1FAFEF74DFBFEF7FA
:103AB000A9FFBDE80840FEF759BD000070470000AF
:103AC000084B1A69920710B508D500241C61202301
:103AD00083F31188FEF77CFB84F31188BDE8104066
:103AE000FEF7B2BF000C0040124B08213220D3F881
:103AF000E82042F00802C3F8E820D3F8102142F091
:103B00000802C3F810210C4AD3F81031D36B43F0EC
:103B10000803D363C722094B9A624FF0FF32DA627F
:103B200000229A615A63DA605A6001225A611A606F
:103B3000FDF720BC004402580010005C000C00405F
:103B4000F8B5514B0024D3F880204FF0FF32C3F872
:103B50008020D3F88010C3F88040D3F88010D3F8C9
:103B60008410C3F88420D3F88410C3F88440D3F8B9
:103B70008410D96F41F0FF4141F4FF0141F4DF416E
:103B800041F07F01D967D96F21F0FF4121F4FF0196
:103B900021F4DF4121F07F01D967D96FD3F8881074
:103BA0006FEA41516FEA5151C3F88810D3F8881079
:103BB000C1F30A01C3F88810D3F88810D3F8901025
:103BC000C3F89020D3F89010C3F89040D3F8901029
:103BD000D3F89410C3F89420D3F89410C3F8944009
:103BE000D3F89410D3F89810C3F89820D3F898100D
:103BF000C3F89840D3F89810D3F88C10C3F88C20F1
:103C0000D3F88C10C3F88C40D3F88C10D3F89C10E8
:103C1000C3F89C20D3F89C20C3F89C40D3F89C3078
:103C200000F0E4F9194B07229A60194ADA60194A40
:103C30001A6105225A60184A536A43F4803353626A
:103C4000C2F88440BFF34F8FD2F8803043F6E0765D
:103C5000C3F3C904C3F34E33A5075B0103EA060EA1
:103C6000284621464EEA0007013900F14040C2F8DB
:103C700074724F1CF6D1203B13F1200FEED1BFF32D
:103C80004F8FBFF36F8FF8BD0044025890ED00E0F6
:103C9000000004301B00080300ED00E00122574B38
:103CA00057491A60574B19609A60574ADA600022E8
:103CB0001A614FF440429A619A699004FCD51A68DF
:103CC00042F480721A60514B1A6F12F4407F04D094
:103CD0004FF480321A6700221A671A6842F0010214
:103CE0001A604A4A134611684907FCD50021116140
:103CF0001A6912F03802FBD1012119604FF080419E
:103D000059605A67424ADA62424A1A611A6842F4B2
:103D100080321A603D4B1A689203FCD53E4A3F49F7
:103D20009A6200225A631963A1F58021DA634B3944
:103D300099635A643A4A1A643A4ADA621A6842F053
:103D4000A8521A60314B1A6802F02852B2F1285F6B
:103D5000F9D1482222219A614FF48862DA61402227
:103D60001A624FF00052DA641A652F4A5A652F4AD8
:103D70009A652F4A11601A6942F003021A61234BB7
:103D80001A6902F03802182AFAD1D3F8DC2042F07E
:103D90000052C3F8DC20D3F8042142F00052C3F8EB
:103DA0000421D3F80421D3F8DC2042F08042C3F888
:103DB000DC20D3F8042142F08042C3F80421D3F878
:103DC0000421D3F8DC2042F00042C3F8DC20D3F811
:103DD000042142F00042C3F80421D3F80421D3F8AF
:103DE000F42042F00202C3F8F420D3F81C2142F080
:103DF0000202C3F81C21D3F81C317047088100511E
:103E000000C000F0004802580200000100440258BF
:103E10000000FF01008890081210200063020701D3
:103E200047040508FD0BFF010010E0000001010040
:103E300000200052084A08B5936811680B4003F04F
:103E40000103936023B1054A13680BB1506898478A
:103E5000BDE80840FEF7F8BD80000058C0270020EC
:103E6000084A08B5936811680B4003F00203936099
:103E700023B1054A93680BB1D0689847BDE8084064
:103E8000FEF7E2BD80000058C0270020084A08B5B0
:103E9000936811680B4003F00403936023B1054A53
:103EA00013690BB150699847BDE80840FEF7CCBDD7
:103EB00080000058C0270020084A08B593681168A0
:103EC0000B4003F00803936023B1054A93690BB1DB
:103ED000D0699847BDE80840FEF7B6BD800000589D
:103EE000C0270020084A08B5936811680B4003F00A
:103EF0001003936023B1054A136A0BB1506A9847C7
:103F0000BDE80840FEF7A0BD80000058C027002093
:103F1000174B10B59C681A68144004F478729A60C4
:103F2000A30604D5134A936A0BB1D06A984760067A
:103F300004D5104A136B0BB1506B9847210604D57A
:103F40000C4A936B0BB1D06B9847E20504D5094A34
:103F5000136C0BB1506C9847A30504D5054A936CBC
:103F60000BB1D06C9847BDE81040FEF76DBD00BFA7
:103F700080000058C02700201A4B10B59C681A68B2
:103F8000144004F47C429A60620504D5164A136D0D
:103F90000BB1506D9847230504D5134A936D0BB1AF
:103FA000D06D9847E00404D50F4A136E0BB1506EE4
:103FB0009847A10404D50C4A936E0BB1D06E984774
:103FC000620404D5084A136F0BB1506F984723045D
:103FD00004D5054A936F0BB1D06F9847BDE81040E8
:103FE000FEF732BD80000058C0270020062108B52A
:103FF0000846FDF7BFF906210720FDF7BBF90621AA
:104000000820FDF7B7F906210920FDF7B3F90621CD
:104010000A20FDF7AFF906211720FDF7ABF90621BD
:104020002820BDE80840FDF7A5B9000008B5FFF756
:1040300087FDFDF775F8FDF747FBFDF71FFDFDF761
:10404000F1FBFFF73BFDBDE80840FFF78FBC000028
:1040500010B501390244904201D1002010BD10F882
:10406000013B11F8014FA342F5D0181B10BD000011
:10407000034611F8012B03F8012B002AF9D17047F0
:10408000121012131211000001105A0003105900EF
:104090000120580003205600E82E00204028002070
:1040A00053544D333248373F3F3F0053544D333222
:1040B000483734332F3735330000000000960000B6
:1040C00000000000000000000000000000000000F0
:1040D0000000000000000000911600087D16000896
:1040E000B9160008A5160008B11600089D160008AC
:1040F0008916000875160008C516000800000000A3
:104100009D17000889170008C5170008B117000897
:10411000BD170008A91700089517000881170008A7
:10412000211800080000000001000000000000004D
:104130006D61696E0000000050410008F02C002005
:10414000E82E0020010000004521000800000000CA
:1041500069646C65000000000200000000000000BF
:10416000C9190008351A00084000400080330020BB
:104170009033002002000000000000000300000057
:1041800000000000791A0008000000001000000084
:10419000A03300200000000001000000000000002B
:1041A00010360020010102004172647550696C6F85
:1041B000740025424F415244252D424C0025534561
:1041C0005249414C250000000D25000875240008C7
:1041D00035190008F124000843000000E041000800
:1041E00009024300020100C032090400000102027A
:1041F000010005240010010524010001042402022D
:104200000524060001070582030800FF09040100D8
:10421000020A0000000705010240000007058102B4
:1042200040000000120000002C42000812011001A2
:104230000200004009124157000201020301000080
:104240000403090425424F4152442500426561732D
:1042500074483700303132333435363738394142DB
:10426000434445460000000000000000E91B000830
:10427000C91E0008751F0008400040004837002094
:10428000483700200100000058370020800000005F
:1042900040010000080000000001000000040000D0
:1042A000080000000001A86A00000000AAAAAAAA4B
:1042B00000011440FFFF00000000000070A70A008A
:1042C0000000000000000000AAAAAAAA0000000046
:1042D000FFFF0000000000000000000000000004DC
:1042E00000000000AAAAAAAA00000000FFDF000048
:1042F00000000000000000000000000000000000BE
:10430000AAAAAAAA00000000FFFF00000000000007
:10431000000000000001000000000000AAAAAAAAF4
:1043200000010000FFFF000000000000000000008E
:104330000000000000000000AAAAAAAA00000000D5
:10434000FFFF00000000000000000000000000006F
:1043500000000000AAAAAAAA00000000FFFF0000B7
:10436000000000000000000000000000000000004D
:10437000AAAAAAAA00000000FFFF00000000000097
:10438000000000000000000000000000AAAAAAAA85
:1043900000000000FFFF000000000000000000001F
:1043A0000000000000000000AAAAAAAA0000000065
:1043B000FFFF0000000000000000000000000000FF
:1043C00000000000AAAAAAAA00000000FFFF000047
:1043D0000000000000000000FF00000000000000DE
:1043E000A04000083F00000050040000AB4000085F
:1043F0003F000000009600000000080004000000DC
:104400004042000800000000000000000000000022
:0C441000000000000000000000000000A0
:00000001FF
